:100000000C9434000C9451000C9451000C94510049
:100010000C9451000C9451000C9451000C9451001C
:100020000C9451000C9451000C9451000C9451000C
:100030000C9451000C9451000C9451000C945100FC
:100040000C9451000C9451000C94AA040C9451008F
:100050000C9451000C9451000C9451000C945100DC
:100060000C9451000C94510011241FBECFEFD8E026
:10007000DEBFCDBF16E0A0E0B1E0ECECFEE102C0D7
:1000800005900D92AC3FB107D9F72BE0ACEFB6E08D
:1000900001C01D92A630B207E1F70E9422040C9421
:1000A000640F0C940000F999FECF92BD81BD60BD34
:1000B000FA9AF99A0895F999FECF92BD81BDF89AFE
:1000C00080B50895EF92FF920F931F93CF93DF9324
:1000D0008C01EB017B01E40EF51ECE15DF0539F036
:1000E0006991C8010E9453000F5F1F4FF6CFDF9147
:1000F000CF911F910F91FF90EF900895EF92FF9293
:100100000F931F93CF93DF938B01040F151FEB0108
:100110007C01E61AF70AC017D10739F0C7018C0F26
:100120009D1F0E945B008993F6CFDF91CF911F91B5
:100130000F91FF90EF9008956F927F928F929F9210
:10014000AF92BF92CF92DF92EF92FF920F931F93E5
:10015000CF93DF93CDB7DEB7C254D1090FB6F89471
:10016000DEBF0FBECDBF6C017B018A0143E050E0D2
:1001700060E071E0C7010E94510C892B09F081C039
:10018000F7018381882309F47CC040E150E070E0EE
:1001900060E0C70104960E94140B23967FAF6EAFF8
:1001A00023976115710509F466C07601F0EEEF0E34
:1001B000F11CF7015081503208F05DC09B0145E011
:1001C00065E270E0C601F6E05F9F800D911D11248D
:1001D0000E944C08F70160816F5F90E080E00E9410
:1001E0005300F701808190E0880F991F42E050E0B2
:1001F000BE016F5B7F4F01960E94620023968FAD18
:1002000023978F9322968FAD22978F93F70180814A
:100210001F928F9384E091E09F938F939E012F5FB5
:100220003F4F69013F932F930E94670C40E450E0D9
:10023000B601C8010E942105F70180818F5F80838C
:100240000FB6F894DEBF0FBECDBFCE5BDF4F0FB64B
:10025000F894DEBF0FBECDBFDF91CF911F910F91FC
:10026000FF90EF90DF90CF90BF90AF909F908F90D6
:100270007F906F90089564E271E0C8010E943D058F
:10028000E4CF44E050E06DE571E0C7010E94510CFD
:10029000892BD1F562E671E0C8010E943D05712C01
:1002A000460130EE830E911C96E0692E21E1A22ECC
:1002B00021E0B22ECE0101967C01F40180817816F6
:1002C000F0F4C601769C800D911D11240E94450812
:1002D0009F938F931F927F92BF92AF92FF92EF9264
:1002E0000E94670C40E450E0B701C8010E9421055C
:1002F00073940FB6F894DEBF0FBECDBFDECF6AE0B9
:10030000C8010E941A05A1CF42E050E06FE872E0F8
:10031000C7010E94510C892BB1F5F7018281882316
:1003200091F1C70102960E942A0CF601E052FF4F9C
:100330002081281728F17C01FF24960146E0849F44
:10034000200D311D1124C9010E940808FF92EF926F
:100350008BE691E09F938F93CE0101967C019F9352
:100360008F930E94670C40E450E0B701C8010E94DF
:1003700021050F900F900F900F900F900F9065CF69
:1003800060E871E07ACF43E050E067EA72E0C701CD
:100390000E94510C892BF1F4F70183818823D1F05D
:1003A000C70103960E942A0CF601E052FF4F2081FC
:1003B000281730F37C01FF24960146E0849F200D2E
:1003C000311D1124C9010E942708FF92EF9280E994
:1003D00091E0C0CF45E050E066EA71E0C7010E94BD
:1003E000510C892B89F5F7018381882369F16CEA27
:1003F00071E0C8010E943D055601F0EEAF0EB11C40
:10040000F501408150E070E060E0C8010E946105A4
:100410006CE2C8010E941A05F12C86E0E82EF50175
:100420008081F81608F06BCFC601FE9C800D911DEF
:1004300011240E94490861E3811101C060E3C801F1
:100440000E941A05F394EBCF4BE150E0B701C801CD
:100450000E9421056FEA71E010CFAF92BF92CF9258
:10046000DF92EF92FF920F931F93CF93DF93CDB75D
:10047000DEB7C054D1090FB6F894DEBF0FBECDBFB2
:100480006C018B017A0142E050E06FE872E0C80134
:100490000E94510C892B49F4C6010E94D80864EED1
:1004A00071E0C7010E943D053FC043E050E067EAAC
:1004B00072E0C8010E94510C892B31F4C6010E94E0
:1004C000050963EF71E0EDCF45E050E063E072E0D5
:1004D000C8010E94510C892BC9F5C6010E94C80AA7
:1004E000082FC6010E94CB0A182FC6010E94C60A17
:1004F0001F920F931F921F931F928F9389E092E098
:100500009F938F938E010F5F1F4F1F930F930E9436
:10051000670C40E450E0B801C7010E9421050FB606
:10052000F894DEBF0FBECDBFC05CDF4F0FB6F894AE
:10053000DEBF0FBECDBFDF91CF911F910F91FF9016
:10054000EF90DF90CF90BF90AF90089543E050E0E0
:100550006AE772E0C8010E94510C892B41F5F8014D
:1005600080E09191992321F08C3139F08F5FF9CFA0
:1005700060E472E08F3008F494CFF801178213869C
:10058000C8010C960E942A0CA82EC80108960E9449
:100590002A0CB82EC80104960E942A0C2A2D4B2D35
:1005A000682FC6010E94130960E372E07ACF47E02A
:1005B00050E062E672E0C8010E94510C892B59F4A8
:1005C000C80108960E942A0C682FC6010E94E708FD
:1005D0006AE672E066CF46E050E067E772E0C80185
:1005E0000E94510C892B59F4C80107960E942A0CCD
:1005F000682FC6010E9427096EE772E052CF47E0DC
:1006000050E06AE872E0C8010E94510C892B39F46D
:1006100061E0C6010E94790962E972E042CF48E0D8
:1006200050E062EA72E0C8010E94510C892B39F453
:1006300060E0C6010E9479096BEA72E032CF4CE1BA
:1006400050E0B801C7010E9421056CEB72E029CF90
:10065000AF92BF92CF92DF92EF92FF920F931F93D0
:10066000CF93DF93CDB7DEB7A0970FB6F894DEBF78
:100670000FBECDBF8C016B015A010E94EB05882390
:1006800001F140E250E0BE016F5F7F4FC8010E9460
:1006900033067C01892BA9F085E0E816F10414F1FA
:1006A00045E050E060E073E0CE0101960E94510CFD
:1006B000892BE9F4A801BE01695F7F4FC6010E9442
:1006C0009C00A0960FB6F894DEBF0FBECDBFDF91A1
:1006D000CF911F910F91FF90EF90DF90CF90BF903F
:1006E000AF90089583E0E816F1040CF441C043E0B4
:1006F00050E066E073E0CE0101960E94510C892B18
:1007000041F4A801BE016B5F7F4FC5010E942D021D
:10071000D8CF85E0E816F1045CF143E050E066EAEA
:1007200071E0CE0101960E94510C892B51F345E0F6
:1007300050E06AE073E0CE0101960E94510C892BD3
:10074000B9F4F12CE12C60E0C7010E9453008FEF57
:10075000E81AF80A81E4E816F104A9F760E173E009
:10076000C8010E943D05F601E052FF4F1082A9CF5B
:1007700089818F3371F084E0E816F10484F044E05D
:1007800050E06FE173E0CE0101960E94510C892B7D
:1007900031F464E273E0C8010E943D0592CF6AEC37
:1007A00076E0F9CFCF92DF92EF92FF920F931F93F3
:1007B000CF93DF9300D0CDB7DEB76C0190E080E03F
:1007C0000E945B00760190EEE90EF11CF701808338
:1007D000813268F010E000E060E0C8010E94530040
:1007E0000F5F1F4F01341105B9F7F701108210E0B8
:1007F00006E0F70180818117D0F0812F90E0880F0B
:10080000991F42E050E0BE016F5F7F4F01960E944A
:100810007E0029813A8145E065E270E0C601109FC3
:10082000800D911D11240E944C081F5FE2CF0F9094
:100830000F90DF91CF911F910F91FF90EF90DF907C
:10084000CF900895CF93DF93CDB7DEB7DA950FB68B
:10085000F894DEBF0FBECDBF82E284B988E68AB9C4
:1008600015B87894CE0193950E9407051F92812CAC
:10087000AA24A394CC24C39483E0E82E08E410E0D7
:1008800027E430E045E450E064E470E0CE018850B5
:100890009F4F0E9456081F92C12C95E0E92E04EB51
:1008A00010E023EB30E041EB50E060EB70E0CE0174
:1008B00080519F4F0E945608CE0188509F4F0E9442
:1008C0009B08CE0180519F4F0E949B08AE01405172
:1008D0005F4FBE0168507F4FCE018E519F4F0E94E7
:1008E000C6088E010F5F1F4F6E0181ECC80ED11C30
:1008F0000F900F907801C8010E9453080A5F1F4FA4
:100900000C151D05C1F780E2F80111928A95E9F7EF
:10091000CF51DF4F1882C15ED040C7010E94D20381
:100920006FED76E0CE0193950E943D05AE014E51EC
:100930005F4FB701CE0193950E942803CE018E51DF
:100940009F4F0E944C0A8FE39FE10197F1F700C08F
:100950000000ECCF1F920F920FB60F9211242F932D
:100960004F935F936F937F938F939F93AF93BF93B7
:10097000EF93FF932091C6008091000790910107AB
:10098000A0910207B09103079370AA27BB278C5F41
:10099000984FFC0120838091000790910107A0915E
:1009A0000207B09103074091FC065091FD0660914B
:1009B000FE067091FF06841B950BA60BB70B8115E5
:1009C0009440A105B10598F480910007909101072A
:1009D000A0910207B09103070196A11DB11D80935C
:1009E000000790930107A0930207B0930307FF91BC
:1009F000EF91BF91AF919F918F917F916F915F9197
:100A00004F912F910F900FBE0F901F9018952AE0D5
:100A1000FC0120831092C50083E38093C40086E02C
:100A20008093C200E1ECF0E088E1808380818068FF
:100A3000808308958091C00085FFFCCF6093C6003D
:100A40000895EF92FF920F931F93CF93DF937C0152
:100A5000EB018B01040F151FC017D10739F0699105
:100A6000662321F0C7010E941A05F6CFDF91CF91CE
:100A70001F910F91FF90EF900895EF92FF920F93C7
:100A80001F93CF93DF937C01EB018B01FE0101905B
:100A90000020E9F73197EC1BFD0BC8018C1B9D0B67
:100AA0008E179F0738F4F80161918F01C7010E94EA
:100AB0001A05ECCFDF91CF911F910F91FF90EF902E
:100AC00008954F925F926F927F929F92AF92BF92E2
:100AD000CF92DF92EF92FF920F931F93CF93DF930A
:100AE000CDB7DEB7C054D1090FB6F894DEBF0FBE44
:100AF000CDBF5C014115510561057105D1F460E37D
:100B00000E941A05C05CDF4F0FB6F894DEBF0FBE1F
:100B1000CDBFDF91CF911F910F91FF90EF90DF90AC
:100B2000CF90BF90AF909F907F906F905F904F90CD
:100B30000895CE0101967C0180E4F70111928A9517
:100B4000E9F7912C77FF0DC0CA0157FF04C0882731
:100B50009927841B950BAC01990F660B770B992491
:100B6000939467010EE310E08AE0482E512C612C2B
:100B7000712C4115510561057105B9F0F1E0CF1AED
:100B8000D1080115110589F001501109CB01BA01F5
:100B9000A30192010E94CD0A942F852F605DF6017A
:100BA00067AFA901692F782FE4CF992039F0F701B9
:100BB000E00FF11F8DE28083015011094FE350E0F7
:100BC000401B510B0F5F1F4FB701600F711FC50115
:100BD0000E94210597CF0F931F930091000710915A
:100BE000010720910207309103074091FC065091C4
:100BF000FD066091FE067091FF0681E040175107E7
:100C00006207730708F080E01F910F9108950E941A
:100C1000EB05882331F18091FC069091FD06A091AF
:100C2000FE06B091FF060196A11DB11D8093FC0642
:100C30009093FD06A093FE06B093FF068091FC06FC
:100C40009091FD06A091FE06B091FF060197A109C3
:100C5000B1099370AA27BB278C5F984FFC01808154
:100C6000089580E008954F925F926F927F928F92E5
:100C70009F92AF92BF92CF92DF92EF92FF920F932B
:100C80001F93CF93DF938C017B01BA0180E090E04A
:100C9000DC01EC018090000790900107A090020712
:100CA000B09003074090FC065090FD066090FE0651
:100CB0007090FF0684189508A608B708881699064C
:100CC000AA06BB0628F1813024E09207A105B105F0
:100CD00009F4A9C02091FC063091FD064091FE0662
:100CE0005091FF064C015D01EFEF8E1A9E0AAE0A8D
:100CF000BE0A280F391F4A1F5B1F33704427552730
:100D00002C5F384FF9013081F8012081321388C0FF
:100D10008090000790900107A0900207B090030711
:100D20004090FC065090FD066090FE067090FF0615
:100D300084189508A608B70888159905AA05BB0563
:100D400008F076C0209781F1570190E080E04B01D8
:100D5000F1E08F1A91086C012FEFC21AD20A8815A0
:100D6000990508F063C0C8010E940706F501819348
:100D70005F01C601CC16DD0671F7EC0CFD1CF70116
:100D800011828091FC069091FD06A091FE06B09123
:100D9000FF060196A11DB11D8093FC069093FD06F0
:100DA000A093FE06B093FF068091FC069091FD068D
:100DB000A091FE06B091FF068C0F9D1FA11DB11DD5
:100DC0009370AA27BB278C5F984FFC019081F80194
:100DD0008081981313C08091FC069091FD06A0912C
:100DE000FE06B091FF060196A11DB11D8093FC0681
:100DF0009093FD06A093FE06B093FF06CE01DF910F
:100E0000CF911F910F91FF90EF90DF90CF90BF9007
:100E1000AF909F908F907F906F905F904F900895CC
:100E2000D501C40136CFC1E0D4E072CF6C01A5CFAB
:100E3000D0E0C0E0B9CFDC011396ED91FC9114979E
:100E400015968C91159721E030E0A90101C0440F5F
:100E50008A95EAF7942F90958081892380838081F9
:100E6000842B8083613009F04DC087EE93E00197B9
:100E7000F1F700C000001396ED91FC9114974081AA
:100E800015968C911597B90102C0660F771F8A9548
:100E9000E2F7CB0180958423808387EB9BE0019769
:100EA000F1F700C000001396ED91FC91149780813A
:100EB00015969C911597A90101C0440F9A95EAF7E0
:100EC000942F9095982390838081842B808387EE44
:100ED00093E00197F1F700C000001396ED91FC91AB
:100EE0001497808115969C9101C0220F9A95EAF77C
:100EF00020952823208387EB9BE00197F1F700C022
:100F00000000089587EB9BE00197F1F700C0000017
:100F10001396ED91FC911497808115969C911597ED
:100F2000A90101C0440F9A95EAF7409548234083F0
:100F300087EE93E00197F1F7B4CFEF92FF920F9312
:100F40001F93CF93DF93EC01EB81FC8120813D81E6
:100F500081E090E0AC0101C0440F3A95EAF7342FEC
:100F60003095322330832081242B2083E7EEF3E079
:100F70003197F1F700C00000EB81FC8120813D81B9
:100F800001C0880F3A95EAF780958223808387EB2A
:100F90009BE00197F1F700C000000FE010E0EE24A5
:100FA000E394F12C29813A81C701002E02C0880FF9
:100FB000991F0A94E2F78223932361E0892B09F4B5
:100FC00060E0CE010E941B07015011090530110598
:100FD00049F7DF91CF911F910F91FF90EF90089506
:100FE000DC011396ED91FC911497208115963C91AC
:100FF00081E090E001C0880F3A95EAF7809582235E
:10100000808387E199E70197F1F700C00000089518
:101010000F931F93CF93DF93EC010AE010E0CE0112
:101020000E949D0761E0CE010E941B0760E0CE0197
:101030000E941B07CE010E94F0070150110979F7A9
:1010400081E08883DF91CF911F910F9108950F93D5
:101050001F93CF93DF93EC010AE010E0CE010E94D2
:101060009D0760E0CE010E941B0761E0CE010E9457
:101070001B07CE010E94F0070150110979F7188271
:10108000DF91CF911F910F910895FC018181928191
:101090000895FC0180810895FC0174836383328389
:1010A000218345830895FC0110820895AF92CF9269
:1010B000EF920F931F93CF93DF93CDB7DEB7FC0171
:1010C000718360833383228315830483C682A7825E
:1010D000DB011C92DA011C928681882331F0208189
:1010E0003181D9018C9180688C938781882331F07C
:1010F00020813181D9018C9180628C932081318152
:10110000D9018C9183608C93DA018C91BE2DB770DC
:10111000EB2EE82ADA01EC92A281B3811C920480C2
:10112000F581E02D1082DF91CF911F910F91EF900B
:10113000CF90AF900895DC01ED91FC918081837098
:1011400080830895CF93DF93EC010E949B088E81EA
:10115000882329F0E881F9818081806880838F81EC
:10116000882329F0E881F981808180628083DF9182
:10117000CF910895DC011296ED91FC916083089562
:10118000DC011496ED91FC9160830895FC0171835C
:1011900060835383428314821682158217821086DD
:1011A0001186128681E0838787E0848715860895FB
:1011B000CF93DF93EC0181E08D87888199810E9434
:1011C000A2088A819B81DF91CF910C94A208CF93D2
:1011D000DF93EC016C836623A9F060E0888199813C
:1011E0000E94C00860E0888199810E94BA0860E08E
:1011F0008A819B810E94C008CE010E94D8081F826C
:101200001E821D82DF91CF910895CF93DF93EC0171
:101210001D86888199810E949B088A819B81DF912C
:10122000CF910C949B08FC01148260874187228730
:10123000338531110AC0620F7727771F460F572F6A
:10124000511D452B11F40C9405090C94D8086150DC
:10125000603108F04BC0E62FF0E0EF5CF64F0C94E5
:10126000EC0A410946094A094E095209550958092B
:101270005B095E095B09620966096A096E09720900
:10128000740920E54FEF60EA0C94130924E14FEF55
:1012900068ECFACF2CE84FEF64EBF6CF20E040E0AB
:1012A0006FEFF2CF2AE04CE3FBCF2EE14EE1F8CF17
:1012B00020E04BE9F5CF20E04FEF0AC02AE04FEFE6
:1012C00067E3E2CF27E040E568E0DECF2FEF40E0C4
:1012D00060E0DACF2FEF4FEF62E3D6CF26E940E5AB
:1012E0006AE0D2CF2CEDE8CF20E0D1CF24E14DE26F
:1012F000D7CFFC0163870895CF93DF93EC018C81F6
:10130000813041F58D819E812F8121111CC0019674
:101310009E838D836D817E816F3F7105B1F481E085
:101320008F83888199810E94C0086D816095888132
:1013300099810E94BA086D8160548A819B81DF91F6
:10134000CF910C94C0080197E3CF6115710549F75F
:101350001F82E7CF823021F58D819E812F8121115F
:1013600018C001969E838D836D817E816E3F21E042
:10137000720789F481E08F837695679588819981DA
:101380000E94C00860E0888199810E94BA0860E0EC
:10139000D4CF0197E7CF6115710571F71F82ECCFAC
:1013A000833069F58D819E812F81211121C00196A5
:1013B0009E838D836D817E8161158FEF7807D1F4D7
:1013C00081E08F8346E0769567954A95E1F78881BD
:1013D00099810E94C0086E81888199810E94BA0813
:1013E0006D817E8153E0769567955A95E1F7A5CF9B
:1013F0000197DECF6115710529F71F82E3CF843095
:10140000F1F56D817E8188819981611520E27207F5
:10141000C8F536E0769567953A95E1F70E94C008E1
:101420006D817E81613080E2780770F088819981DA
:10143000611520E4720760F5705226E07695679595
:101440002A95E1F70E94BA086D817E81613080E4BF
:10145000780768F064E0769F612D7727112484E196
:10146000689F602D11248A819B810E94C0088D8114
:101470009E818F3F980719F001969E838D83DF919F
:10148000CF910895672F6695669566956058C6CF8B
:10149000672F66956058D6CFCF93DF93EC010E94FB
:1014A0007C098C8181116FC08B85882309F45FC012
:1014B0008D819E8101969E838D839C8501C0880FBE
:1014C0009A95EAF781115FC098B588858917B1F0C0
:1014D00068B528B5281B330B81E090E0121613067F
:1014E00014F090E080E0232F221F2227221F821B6E
:1014F0009109681B888199810E94C00897B58985E8
:101500008917B1F067B527B5281B330B81E090E050
:101510001216130614F090E080E0232F221F2227DA
:10152000221F821B9109681B888199810E94BA0839
:101530009091B4008A85891731F16091B4002091AF
:10154000B400281B330B81E090E01216130614F050
:1015500090E080E0232F221F2227221F821B910967
:10156000681B8A819B81DF91CF910C94C0086985AB
:10157000888199810E94BA086885888199810E9432
:10158000C0086A85EECFDF91CF91089588B50895A0
:101590008091B400089587B50895052E97FB1EF439
:1015A00000940E94E40A57FD07D00E94F20A07FC4B
:1015B00003D04EF40C94E40A509540953095219553
:1015C0003F4F4F4F5F4F089590958095709561956F
:1015D0007F4F8F4F9F4F0895EE0FFF1F0590F4919F
:1015E000E02D0994A1E21A2EAA1BBB1BFD010DC020
:1015F000AA1FBB1FEE1FFF1FA217B307E407F507C3
:1016000020F0A21BB30BE40BF50B661F771F881F9E
:10161000991F1A9469F760957095809590959B0134
:10162000AC01BD01CF010895A0E0B0E0EAE1FBE02C
:101630000C941F0F5C016B017A016115710519F0A3
:10164000FB0191838083E114F10429F0C701029723
:10165000839708F0E5C0E5012196F5011081812FFF
:1016600090E00E94480C892B11F05E01F4CF1D32EE
:1016700029F42196F501118101E007C01B3221F404
:10168000E5012296F501118100E0E114F10409F170
:10169000F0E1EF16F10429F43FC010E3E114F10486
:1016A00021F128E0E216F10401F154F4E2E0EE1633
:1016B000F10421F5812C912CA12CB0E4BB2E3EC06D
:1016C000FAE0EF16F10439F020E1E216F104B1F48A
:1016D00030C0103319F1FAE0EF2EF12CACEC8A2E69
:1016E000982CA82CACE0BA2E29C078E0E72EF12C7B
:1016F000812C912CA12CE0E1BE2E20C060E070E096
:1017000080E090E897010F2C000C440B550B0E94D1
:10171000F20A49015A0112C0103359F488818F7DB1
:10172000883509F0BACF19812296026080E1E82E4F
:10173000F12C812C912CA12C68E0B62E40E060E0C9
:1017400070E0CB0127010F2C000C66087708FE0122
:1017500050ED352E310E29E0231570F42FEB210FBB
:101760002A3118F439EC332E06C02FE9210F2A3123
:1017700018F529EA322E310E232D30E02E153F05C3
:10178000DCF447FD16C086169706A806B90670F069
:10179000A30192010E94030F630D711D811D911D14
:1017A00061307105810520E8920710F04FEF01C00C
:1017B00041E021961081CBCF202F2170C114D1049C
:1017C00071F0442329F02197F601D183C08307C02B
:1017D00001FF19C02297F601D183C08314C047FFCF
:1017E00012C0222329F060E070E080E090E804C09D
:1017F0006FEF7FEF8FEF9FE722E230E03093050B32
:101800002093040B09C0222381F090958095709558
:1018100061957F4F8F4F9F4F462F372F282F12C034
:1018200040E030E020E090E00DC097FFF5CF82E28D
:1018300090E09093050B8093040B6FEF7FEF8FEF99
:101840009FE7EACF642F732F822FCDB7DEB7E1E198
:101850000C943B0FFC0188279927E89421912032B2
:10186000E9F3293010F02E30C8F32B3241F02D323D
:1018700039F4689404C00E945F0C820F911D21917D
:1018800020532A30C0F31EF4909581959F4F089500
:1018900091110C945C0E803219F089508550C8F774
:1018A0000895FB01DC014150504030F08D910190D2
:1018B000801919F40020B9F7881B990B08957AE074
:1018C000979F902D879F802D910D11240895AEE054
:1018D000B0E0EDE6FCE00C942C0F0D891E8986E04B
:1018E0008C831A8309838FEF9FE79E838D83AE01DC
:1018F000475E5F4F6F89788DCE0101960E94890CFB
:10190000EF81F885E00FF11F10822E96E4E00C9431
:10191000480FACE0B0E0EFE8FCE00C941E0F6C0167
:101920007B018A01FC0117821682838181FFBEC17F
:10193000CE0101964C01F6019381F70193FD85914B
:1019400093FF81917F01882309F4ACC1853239F47A
:1019500093FD859193FF81917F01853229F4B60132
:1019600090E00E94750EE7CF512C312C20E0203200
:10197000A0F48B3269F030F4803259F0833269F48C
:1019800020612CC08D3239F0803339F4216026C0BB
:101990002260246023C0286021C027FD27C030EDCD
:1019A000380F3A3078F426FF06C0FAE05F9E300D1B
:1019B0001124532E13C08AE0389E300D1124332E8B
:1019C00020620CC08E3221F426FD6CC1206406C05A
:1019D0008C3611F4206802C0883641F4F70193FD7B
:1019E000859193FF81917F018111C1CF982F9F7DB8
:1019F0009554933028F40C5F1F4F9FE399830DC0DB
:101A0000833631F0833771F0833509F05BC022C033
:101A1000F801808189830E5F1F4F44244394512C29
:101A2000540115C03801F2E06F0E711CF801A0805E
:101A3000B18026FF03C0652D70E002C06FEF7FEF1D
:101A4000C5012C870E946A0E2C0183012C852F77FB
:101A5000222E17C03801F2E06F0E711CF801A08031
:101A6000B18026FF03C0652D70E002C06FEF7FEFED
:101A7000C5012C870E945F0E2C012C852068222E28
:101A8000830123FC1BC0832D90E048165906B0F457
:101A9000B60180E290E00E94750E3A94F4CFF50111
:101AA00027FC859127FE81915F01B60190E00E949D
:101AB000750E31103A94F1E04F1A51084114510457
:101AC00071F7E6C0843611F0893639F5F80127FF41
:101AD00007C060817181828193810C5F1F4F08C0B4
:101AE00060817181072E000C880B990B0E5F1F4FD0
:101AF0002F76722E97FF09C090958095709561950D
:101B00007F4F8F4F9F4F2068722E2AE030E0A40154
:101B10000E94A50EA82EA81844C0853729F42F7E50
:101B2000B22E2AE030E025C0F22FF97FBF2E8F368B
:101B3000C1F018F4883579F0B5C0803719F08837CE
:101B400021F0B0C02F2F2061B22EB4FE0DC08B2D1E
:101B50008460B82E09C024FF0AC09F2F9660B92E5A
:101B600006C028E030E005C020E130E002C020E1FE
:101B700032E0F801B7FE07C06081718182819381F4
:101B80000C5F1F4F06C06081718180E090E00E5FA6
:101B90001F4FA4010E94A50EA82EA818FB2DFF77A9
:101BA0007F2E76FE0BC0372D3E7FA51450F474FEB9
:101BB0000AC072FC08C0372D3E7E05C0BA2C372DF6
:101BC00003C0BA2C01C0B52C34FF0DC0FE01EA0DD4
:101BD000F11D8081803311F4397E09C032FF06C0C7
:101BE000B394B39404C0832F867809F0B39433FD83
:101BF00013C030FF06C0B31498F43A0C532C5B1892
:101C000010C0B31470F4B60180E290E03C870E94EB
:101C1000750EB3943C85F5CFB31418F43B1802C08D
:101C20005A2C312C34FF12C0B60180E390E03C877F
:101C30000E94750E3C8532FF17C031FD03C088E756
:101C400090E002C088E590E0B6010CC0832F867852
:101C500059F031FF02C08BE201C080E237FD8DE216
:101C6000B60190E00E94750EA51438F4B60180E329
:101C700090E00E94750E5A94F7CFAA94F401EA0DF1
:101C8000F11D8081B60190E00E94750EA110F5CF84
:101C9000332009F450CEB60180E290E00E94750E28
:101CA0003A94F6CFF6018681978102C08FEF9FEFBD
:101CB0002C96E2E10C943A0F992788270895FC01AD
:101CC0000590615070400110D8F7809590958E0F67
:101CD0009F1F0895FC016150704001900110D8F7DA
:101CE000809590958E0F9F1F08950F931F93CF930C
:101CF000DF93182F092FEB018B8181FD03C08FEF3C
:101D00009FEF1EC082FF0FC02E813F818C819D817D
:101D10002817390774F4E881F981CF010196998376
:101D20008883108306C0E885F985812F0995892B62
:101D300031F78E819F8101969F838E83812F902F13
:101D4000DF91CF911F910F910895FA01AA272830B2
:101D500051F1203181F1E8946F936E7F6E5F7F4F78
:101D60008F4F9F4FAF4FB1E03ED0B4E03CD0670FF4
:101D7000781F891F9A1FA11D680F791F8A1F911D47
:101D8000A11D6A0F711D811D911DA11D20D009F497
:101D900068943F912AE0269F11243019305D3193D9
:101DA000DEF6CF010895462F4770405D4193B3E0C2
:101DB0000FD0C9F7F6CF462F4F70405D4A3318F069
:101DC000495D31FD4052419302D0A9F7EACFB4E01A
:101DD000A6959795879577956795BA95C9F70097D2
:101DE0006105710508959B01AC010A2E0694579573
:101DF000479537952795BA95C9F7620F731F841FCA
:101E0000951FA01D0895DB018F939F930E94130FD0
:101E1000BF91AF91A29F800D911DA39F900DB29F86
:101E2000900D112408950E94550FA59F900DB49F09
:101E3000900DA49F800D911D112408952F923F9223
:101E40004F925F926F927F928F929F92AF92BF92CA
:101E5000CF92DF92EF92FF920F931F93CF93DF9376
:101E6000CDB7DEB7CA1BDB0B0FB6F894DEBF0FBED3
:101E7000CDBF09942A88398848885F846E847D8420
:101E80008C849B84AA84B984C884DF80EE80FD8022
:101E90000C811B81AA81B981CE0FD11D0FB6F89498
:101EA000DEBF0FBECDBFED010895A29FB001B39F6D
:101EB000C001A39F700D811D1124911DB29F700D53
:0C1EC000811D1124911D0895F894FFCF9E
:101ECC006164640052656C6179207361766564218C
:101EDC00204E554D4245523A2025752049443A2012
:101EEC0025580A0055736167653A2072656C6179F3
:101EFC0020616464205B69645D202020205B696440
:101F0C005D206265696E67206120313662697420DC
:101F1C00686578206E756D6D6265720A006C697308
:101F2C00740052656C6179733A0A0052454C415900
:101F3C003A202575207475726E6564206F6E0A00E8
:101F4C004E6F2073757463682052656C61790A005A
:101F5C0052454C41593A202575207475726E656452
:101F6C00206F66660A007374617465005354002018
:101F7C006973206E6F7420612076616C69642073C4
:101F8C007562636F6D6D616E643A2072656C617918
:101F9C00205B6164642F6C6973742F6F6E2F6F6696
:101FAC00665D0A00524742206C6967687473206F43
:101FBC006E0A00524742206C6967687473206F6622
:101FCC00660A007072696E740043757272656E7485
:101FDC00205247422076616C7565733A0A523A205A
:101FEC00257520473A20257520423A2025750A0090
:101FFC00536574205247422076616C7565730A00F4
:10200C0055736167653A2072676220736574205B53
:10201C005252525D205B4747475D205B4242425D16
:10202C000A007061747465726E005365742050619F
:10203C00747465726E0A0070726573657400536512
:10204C0074205072657365740A0066616465206F54
:10205C006E005475726E6564206F6E204661646507
:10206C000A0066616465206F6666005475726E6561
:10207C0064206F666620466164650A0020697320DF
:10208C006E6F7420612076616C6964207375626375
:10209C006F6D6D616E643A20726762205B2F6F6E9C
:1020AC002F6F66662F7072696E742F7365742F7044
:1020BC0061747465726E2F7072657365745D0A005D
:1020CC0072656C617900726762006572617365009C
:1020DC00454550524F4D206572617365640A006826
:1020EC00656C7000417661696C61626C6520436F50
:1020FC006D6D616E64733A200A2020202020202010
:10210C0020202020202020202068656C702020209A
:10211C0020202020202020202020202020202020B3
:10212C00202020203A202053686F77207468697330
:10213C002070726F6D7074200A20202020202020C7
:10214C0020202020202020202072656C61792061C5
:10215C006464205B69645D202020202020202020E6
:10216C00202020203A202041646420576972656C3D
:10217C006573732052656C61790A20202020202021
:10218C002020202020202020202072656C617920C6
:10219C006C697374202020202020202020202020F7
:1021AC0020202020203A20205072696E74206C6907
:1021BC007374206F6620736176656420576972654D
:1021CC006C6573732052656C617973200A20202032
:1021DC002020202020202020202020202072656C10
:1021EC006179205B6F6E2F6F66665D205B6E6E5D36
:1021FC0020202020202020203A20205475726E2090
:10220C006F6E2F6F6666206E74682072656C6179D4
:10221C000A202020202020202020202020202020C8
:10222C002072656C617920737461746520202020A4
:10223C002020202020202020202020203A20204751
:10224C0065742066756C6C206D616368696E6520C1
:10225C007265616461626C652072656C6179207372
:10226C00746174650A20202020202020202020204A
:10227C0020202020206572617365202020202020E2
:10228C002020202020202020202020202020202042
:10229C003A2020457261736520657070726F6D0A0B
:1022AC002020202020202020202020202020202022
:1022BC00726762205B6F6E2F6F66665D2020202038
:1022CC0020202020202020202020203A202054755F
:1022DC00726E206F6E2F6F666620524742206C65BF
:1022EC0064732061742063757272656E74207661FC
:1022FC006C75652E0A2020202020202020202020F4
:10230C002020202020726762207072696E74202059
:10231C0020202020202020202020202020202020B1
:10232C003A20205072696E742063757272656E74F7
:10233C00205247422076616C75652E0A20202020A1
:10234C0020202020202020202020202072676220A6
:10235C00736574205B5252525D205B4747475D208A
:10236C005B4242425D20203A202053657420524744
:10237C00422076616C75652C207061747465726E88
:10238C00206D75737420626520302E0A2020202069
:10239C002020202020202020202020207267622056
:1023AC007061747465726E205B69645D20202020FE
:1023BC00202020202020203A2020524742207061EB
:1023CC00747465726E0A202020202020202020208A
:1023DC002020202020207267622070726573657443
:1023EC00205B69645D2020202020202020202020DC
:1023FC00203A2020736574207072657365742063B5
:10240C006F6C6F720A20202020202020202020209A
:10241C0020202020207267622066616465205B6F3B
:10242C006E2F6F66665D202020202020202020202B
:10243C003A20207475726E20436F6C6F7266616403
:10244C0065206F6E206F72206F66660A2020202038
:10245C002020202020202020202020207665727330
:10246C00696F6E202020202020202020202020207A
:10247C00202020202020203A20205072696E7420C9
:10248C0056657273696F6E2E0A004E6F7420612050
:10249C0076616C696420636F6D6D616E640A0052C5
:1024AC004742436F6E74726F6C6C65722076302E7F
:0C24BC0034207374617274696E670A004A
:00000001FF
